:020000040000FA
:200000000C94C7000C947A040C94E4000C94E4000C94E4000C94E4000C94E4000C94E40043
:200020000C94E4000C94E4000C94E4000C94E4000C94E4000C94E4000C94E4000C94E400A0
:200040000C945B080C94E4000C94E4000C94E4000C94E4000C94E4000C94E4000C94E40001
:200060000C94E4000C94E40034316439333861382D366638612D313165352D613435652D5E
:2000800030303162666361336335393300000000010102030304050506070708090A0A0BB0
:2000A0000C0D0D0E0F1011121213141516171818191A1B1C1D1E1F2021212223242526271E
:2000C00028292A2B2C2D2E2F303132333435363738393A3B3C3D3E3F40414243454647482C
:2000E000494A4B4C4D4E4F5051535455565758595A5B5D5E5F6061626364666768696A6BC5
:200100006C6E6F7071727375767778797A7C7D7E7F80818384858687898A8B8C8D8F90910C
:200120009294959697989A9B9C9D9FA0A1A2A4A5A6A7A9AAABACAEAFB0B1B3B4B5B6B8B90E
:20014000BABBBDBEBFC1C2C3C4C6C7C8CACBCCCDCFD0D1D3D4D5D7D8D9DADCDDDEE0E1E2DB
:20016000E4E5E6E8E9EAECEDEEF0F1F2F4F5F6F8F9FAFCFDFEFFFFFFFFFFFFFFFFFFFFFFC5
:20018000FFFFFFFFFFFFFFFFFFFFFFFFFF0011241FBECFEFD4E0DEBFCDBF12E0A0E0B1E0BC
:2001A000E8E3FCE102C005900D92AA31B107D9F724E0AAE1B2E001C01D92AE3BB207E1F733
:2001C0000E94670C0C941A0E0C94000001978430910580F428E3289FD001299FB00D1124EF
:2001E000A654BD4FE6E7F2E001900D922A95E1F70C948E08089528E3E0E0F1E0A6E7B2E005
:2002000001900D922A95E1F7019784309105B8F448E3489F9001499F300D1124F901E65458
:20022000FD4FD901A255BD4F1C968C918F3F51F088E3A6E7B2E001900D928A95E1F780E0A6
:2002400090E008958FEF9FEF0895FC0185858823A1F00E9484088823A1F080911A029091ED
:200260001B02019690931B0280931A0206974CF00E94A80B81E090E0089510921B0210925E
:200280001A0280E090E008959B01285F3F4F90E8492F4823FB014193BF019695E217F3071B
:2002A000B9F708951F93CF93DF9320E030E0EB01C20FD31F241735078CF4DC011896FC012D
:2002C00090E080E811911111982B8695EA17FB07C9F798832F5F3F4FCF01E9CFDF91CF9152
:2002E0001F910895FF920F931F93CF93DF93CDB7DEB7A0970FB6F894DEBF0FBECDBFFC0164
:200300008B0181E021819381291301C080E0898381E025819781291301C080E08A8381E0E7
:2003200021859385291301C080E08B8381E025859785291301C080E08C8381E021A593A5A2
:20034000291301C080E08D8381E025A597A5291301C080E08E8381E021A993A9291301C0F7
:2003600080E08F8381E025A997A9291301C080E0888719861A8681E021899389291301C0CD
:2003800080E08B8781E025899789291301C080E08C8781E0218D938D291301C080E08D87AC
:2003A00081E0258D978D291301C080E08E8781E021A193A1291301C080E08F8781E025A1A3
:2003C00097A1291301C080E0888B21AD95ADDF01A05CBF4F11968C91119713963C91831303
:2003E00001C0892FDF01AC5BBF4F1196FC90119713969C91F91201C0F82EDF01A85BBF4FFB
:2004000011969C91119713968C91981301C0922FE45BFF4F81812381821301C0892FBE016D
:200420006F5E7F4F0E944401BE01675E7F4F8F2D80950E94440144E050E0B801CE010196BD
:200440000E945201A0960FB6F894DEBF0FBECDBFDF91CF911F910F91FF900895F8940E94B0
:200460006F08E0E0FCE109940895CF93C82F823008F4B1C080912D02823509F0ACC0909139
:200480002E02933009F46EC028F4913069F008F4A0C02DC0993F09F48EC09F3F09F496C06B
:2004A000943009F098C07BC088E2EDE2F2E0DF011D928A95E9F710922D028091B6028093A6
:2004C0002E028091B70280932F028091B802809330028091B902809331029093360266E11A
:2004E00072E087E392E00E94EB0D8EE075C0C43008F471C020912F0280913002253008F0FE
:200500006AC030E02115310559F02150310998E3929FF001939FF00D1124E654FD4F02C0F8
:20052000E6E7F2E090E0009721F488E380932D0234C08130910549F480E2ADE2B2E00190C7
:200540000D928A95E1F780E247C0029709F043C0B09688E1ADE2B2E001900D928A95E1F710
:2005600088E13AC0C430B8F180912F02813059F048E350E06FEF70E086E792E00E94E40DC4
:2005800086E792E002C086E992E04C2F50E04450510960E372E00E94DB0D81E01DC0C230F1
:2005A000D1F020912F02822F90E00197049738F420931C0208C080911C02882321F081E033
:2005C00080932D0209C010922D02E7CF0E942E0202C08C2F01C080E0CF910895009741F054
:2005E00028E0E5E2F2E0DC0101900D922A95E1F788E0E5E2F2E0ADE1B2E001900D928A9546
:20060000E1F708958091380190913901892B31F0109239011092380181E0089548E050E0DE
:200620006DE172E085E292E00E94CE0D0895CF93DF93CDB7DEB728970FB6F894DEBF0FBEC0
:20064000CDBFFE01319688E0DF011D928A95E9F7698180E090E020E830E0DC01A653BC4F9F
:200660004C91442341F0A901082E02C0559547950A94E2F701C040E0462B019688309105EF
:2006800011F0642FEACF49836A8180E090E020E830E0DC01AE52BC4F4C91442341F0A90167
:2006A000082E02C0559547950A94E2F701C040E0462B01968830910511F0642FEACF4095AC
:2006C0004A836B8180E090E020E830E0DC01A652BC4F4C91442341F0A901082E02C0559598
:2006E00047950A94E2F701C040E0462B01968830910511F0642FEACF4B836C8180E090E098
:2007000020E830E0DC01AE51BC4F4C91411108C0A901082E02C0559547950A94E2F701C043
:2007200040E0462B01968830910511F0642FEACF4C836D8180E090E020E830E0DC01A6517D
:20074000BC4F4C91442341F0A901082E02C0559547950A94E2F701C040E0462B0196883099
:20076000910511F0642FEACF40954D836E8180E090E020E830E0DC01AE50BC4F4C914423F0
:2007800041F0A901082E02C0559547950A94E2F701C040E0462B01968830910511F0642F7E
:2007A000EACF40954E833F8180E090E041E0DC01A354BC4F2C91222339F0242F082E01C0D5
:2007C000220F0A94EAF701C020E0322B01968530910569F78091C303882311F080E201C063
:2007E00080E0382B8091C403882311F080E401C080E0382B8091C503882311F080E801C01C
:2008000080E0382B3F83288580E090E051E0DC01AA53BC4F4C91442339F0452F082E01C0E8
:20082000440F0A94EAF701C040E0242B01968430910569F72887A5E2B2E0CE01079641916F
:200840004D93E817F907D9F730932B0220932C0228960FB6F894DEBF0FBECDBFDF91CF9143
:200860000895CF93DF93CDB7DEB729970FB6F894DEBF0FBECDBF198661E070E0CE01099649
:200880000E9460098831B9F487EC90E00197F1F700C0000080E4898383E08A831B8263E004
:2008A00070E0CE0101960E946009803421F40E94170380E001C081E029960FB6F894DEBFC3
:2008C0000FBECDBFDF91CF91089581E00E94310491E0811190E0892F08958FB7F894219AC5
:2008E00029983B9843988FBF81E00C9431048AE391E008951F921FB64F930F931F93EF934C
:20090000FF937F93AF93BF93ADE2B2E00027E5E2F5E049B14470440F440F440F440F440F6E
:20092000042B49B14470E9F31AE01A9521F049B14470D9F701C0099416E01A95F1F749B1E1
:200940004470440F440F440F440F042B49B14470E9F31AE01A9521F049B14470D9F701C0E5
:20096000099416E01A95F1F749B14470440F440F440F042B49B14470E9F31AE01A9521F033
:2009800049B14470D9F701C0099416E01A95F1F749B14470440F440F042B49B14470E9F3E1
:2009A0001AE01A9521F049B14470D9F701C0099416E01A95F1F749B14470440F042B49B1EA
:2009C0004470E9F31AE01A9521F049B14470D9F701C0099416E01A95F1F749B14470042B87
:2009E00049B14470E9F31AE01A9521F049B14470D9F701C0099416E01A95F1F749B144709C
:200A00004695042B49B14470E9F31AE01A9521F049B14470D9F701C0099416E01A95F1F71F
:200A200049B1447046954695042B49B14470E9F30D931AE01A9521F049B14470D9F701C000
:200A4000099415E01A95F1F761CF0DE2A01B91F1A13011F10F921F922F933F934F935F9384
:200A60006F937F938F939F93AF93BF93FF938A2F1124E5E3F2E00995082FFF91BF91AF916B
:200A80009F918F917F916F915F914F913F912F911F900F901FD00EC0ADE2B2E00C9101309C
:200AA00011F422D007C0003019F00F3F09F002C016D000C041E0E0E6F2E04083E09ABF914A
:200AC000AF917F91FF91EF911F910F914F911FBE1F901895EDE2F2E0702F13D00895EDE5BB
:200AE000F2E073E00ED00895E1E6F2E07081772319F4E5E5F2E002C0E9E5F2E074E001D002
:200B000008953F937723D9F1772359F17A95019110E8302F312381F40000529A4FE04A9563
:200B2000F1F700005298169579F3000000000000000000000000EDCF529A44E04A95F1F739
:200B40000000000052984AE04A95F1F7000000001695D1F20000000000000000000000004C
:200B6000D8CF00000000000000000000000000000000529A44E04A95F1F7000052983F913D
:200B80000895FC0120812F3F59F0332727FD30952617370719F4FC01418308950296F1CFE2
:200BA0000895FC012081223011F48181089580E00895FC018081833031F0843059F0813087
:200BC00069F4818108958281918187FD05C098172CF006C091818281891714F480E0089570
:200BE00081E00895CF92DF92EF92FF920F931F93CF93DF938C017B016A019A012C5F3F4FC3
:200C0000F90134978081882319F1F9013197808132978083F3CFF8019181E601F4E09F02A1
:200C2000C00DD11D112498819230B9F0933001F1913061F4970144E08402200D311D112483
:200C4000C9010E94D9059981982B99830E5F1F4FF80180818F3FF9F619C0F70194E08902EF
:200C6000E00DF11D11248081823081F781810CC0F70124E08202E00DF11D1124CF010E9429
:200C8000D905882319F38A818983E0CFDF91CF911F910F91FF90EF90DF90CF900895FC0163
:200CA000208120582093630281818058809362020895E091B902E13029F020E935E640E07B
:200CC00050E004C028EA31E640E050E09091B702992341F09CE0E13039F020E335E740E0EB
:200CE00050E006C090E004C028E431E740E050E06058A62FBB27A7FDB095A81BB10987FDFD
:200D0000B3959923F9F01A161B0654F4892F992787FD9095A817B9079CF0A81BB90B12C0C8
:200D2000109781F0892F992787FD909566277727681B790B6A177B071CF0A80FB91F02C0E8
:200D4000A0E0B0E0E33049F00E94990D20E03DE740E050E00E94640DD901A2388FEFB80777
:200D600034F0A038B1052CF0AFE7B0E002C0A1E8BFEFCD0108952F923F924F925F926F92B6
:200D80007F928F929F92AF92BF92CF92DF92EF92FF920F931F93CF93DF93CDB7DEB72A9778
:200DA0000FB6F894DEBF0FBECDBFD62E5A8349833C832B839091B902933091F4682F809106
:200DC00063020E945906182F6D2D809162020E945906E981FA811083EB81FC81808387C0AB
:200DE000913039F0412C512C3201539400E510E007C0412C92E0592E612C712C0FE710E0F3
:200E0000682F809163020E9459067C016D2D809162020E9459069A8789879C0197FF03C010
:200E20003195219531091701F7FE04C0222433242E183F084701AA2497FCA094BA2C30E02E
:200E4000D7010E94920DA30192010E94640D2D833E834F83588729853A856901EE24D7FC51
:200E6000E094FE2C222D30E0A985BA850E94920DA30192010E94640DC20ED31EE41EF51EA7
:200E800088279927801B910BAA2797FDA095BA2F2D813E814F815885820E931EA41EB51E39
:200EA00088169906AA06BB0614F44C015D01222717FD2095322F081519052A053B0514F4AC
:200EC000480159018C159D05AE05BF0534F40C151D052E053F052CF002C06C017D01970172
:200EE0008601E981FA818082EB81FC8100832A960FB6F894DEBF0FBECDBFDF91CF911F9191
:200F00000F91FF90EF90DF90CF90BF90AF909F908F907F906F905F904F903F902F90089572
:200F20000F931F93CF93DF938C01EB01DC0116968C9116978071898316968C911697887052
:200F40008D8316968C9116978078898716968C91169781708D8716968C9116978072898B0C
:200F600016968C91169780748D8B13968C9113978058898F13968C91139780588D8F129683
:200F80008C911297805889A312968C91129780588DA317968C911797817089A717968C91AE
:200FA000179782708DA717968C911797887089AB17968C91179784708DAB9B01235C3F4F6C
:200FC000AB01475C5F4F11966C9111978C910E94BB06FE01E05CFF4FD80116968C91169770
:200FE00084708183349616968C911697827081838DAD349681833496818389AD34968183E9
:2010000034968183349614968C91149780588183349615968C9180588183349689A1818384
:201020003496898D8183DF91CF911F910F9108958093640208952998219A089520916402C9
:20104000222331F021E0892B09F020E0822F90E0892B11F0299A089529980895CF93DF9314
:20106000EC0181E090E00E941E082FEF87EE93E0215080409040E1F700C0000080E090E07B
:201080000E941E082FEF87EE93E0215080409040E1F700C000002197209719F7DF91CF919A
:2010A00008958AE090E00E942E081092640280E090E00C941E0878941F920F920FB60F927F
:2010C00011248F93809165028C3318F48F5F809365028F910F900FBE0F901F901895EEE6B3
:2010E000F0E080818E7F80830895EEE6F0E0808181608083089514BC85E085BD81E0809361
:201100006E00109265020895809165028C3320F01092650281E0089580E008954CE051E013
:2011200060E070E08EEA92E00C94020E88E0EEE0F2E0AEEAB2E001900D928A95E1F710928A
:20114000B6021092B7021092B80282E08093B90240E051E06FEF70E08AEB92E00E94E40D77
:201160000C948E084CE051E060E070E08EEA92E00E94F20D48E050E06EE072E08EEA92E0DF
:201180000E94CE0D009721F00E94960881E090E008958091B9028F5F843008F081E08093A2
:2011A000B9028091B902813019F48093B80208951092B802089581E09091B702911180E04A
:2011C0008093B7020C948E088093B6020C948E081092800083E0809381001092850010922A
:2011E00084001092670286ED96E090936902809368020895A89B08C0A89A86ED96E0909376
:2012000069028093680229C02091840030918500293E83E0380780F1273D86E0380728F1E6
:20122000A6E0B0E00E94830D27E030E040E050E00E94640D30936902209368028091680226
:2012400090916902883E934030F486ED96E09093690280936802109266021092850010927E
:201260008400A89A10926702089586ED96E09093690280936802E2CF809166028F5F8093E1
:201280006602893050F381E090E0E1CF8091670281110FC020918400309185008091680298
:2012A000909169022817390720F081E080936702089580E008953B984398249A2C980895CF
:2012C0000F931F93CF93DF93662309F454C07727A0E0B0E040E050E09D0146175707ACF455
:2012E000189610E8FC01E40FF51F00810123E901C654DC4F08832F5F3F4F16952A173B079B
:20130000A1F74F5F5F4FD901E7CFEAEBF3E0CF93DF93EF93FF930191002311F069F41BC0CB
:2013200000003B9A1DE014D03B980000000000000000119781F70FC03B9A12E0000008D096
:201340003B9819E005D000000000119721F703C01A95F1F7089500000000FF91EF91DF91B5
:20136000CF913B9A12E00000F3DF3B980FEF0A9511F0339BFCCFEAEBF3E0EF93FF93442743
:2013800000270395A1F03399FCCF08C00BE4039572F03399FCCF439551F001930BE40395EA
:2013A00032F0339BFCCF439511F00193EFCFFF91EF91842F90E00097C1F040FF16C0DF01D7
:2013C0009D017081618151E0761708F050E05D9332965A2F521B5417A0F32AE12A95F1F758
:2013E00000C001979595879502C080E090E0DF91CF911F910F910895CF93DF931F92CDB7F7
:20140000DEB7198261E070E0CE0101960E9460090097F1F04897F9F48091BE03811188E08A
:201420009091BF03911184609091C003911182609091C103911181608A3038F4883070F471
:20144000853049F481E090E00BC08B3039F003C080E090E005C083E090E002C082E090E05B
:201460000F90DF91CF9108958FEF99EF0197F1F700C00000E0916C02F0916D020484F58549
:20148000E02D80E00995E0916C02F0916D020684F785E02D0995882339F3E0916C02F0918A
:2014A0006D020088F189E02D8EE692E009956EE471E08EE692E00E94900791E080E02091E6
:2014C0004F01211101C090E0292F382F809153018111226080918F018111246080919301C5
:2014E00081112860809157018111206180915F0181112062809163018111206480917701BD
:201500008111206880917B018111316080917F0181113260809183018111346080915B0124
:201520008111386060916A0270916B02622773274CE050E081E090E0FC01E623F723EF2B2C
:2015400051F0FC01E223F323EF2B29F030936B0220936A020895880F991F41505109411583
:20156000510551F730936B0220936A027DCFEF92FF920F931F93CF93DF9300D01F92CDB7F3
:20158000DEB78B018032910519F07B0120E81EC0FB01808191818F3FFFEF9F0709F454C0F5
:2015A0000196FB014EC089309105A4F482309105A1F184309105A9F1019761F129834A8382
:2015C0005B830E94340A5B814A8129818830910551F72BC08032910561F18115F8E09F07CD
:2015E00099F1409759F7203841F0822F90E0F701918380837A0120E8E1CFF8018081918142
:201600008F3FFFEF9F0701F10196F801918380837A01D4CF220F220FD1CF220F220F2F5FBF
:20162000CDCF220F220F2E5FC9CF220F220F2D5FC5CFE016F10641F0203849F0822F90E035
:20164000F7019183808303C08FEF9FEF02C080E090E00F900F900F90DF91CF911F910F911D
:20166000FF90EF90089581E090E00E942E080E94340A811522E09207B9F04CF480389105CE
:2016800081F081159140D1F482E090E012C0811524E0920761F08115984081F480E090E0D2
:2016A00008C081E090E005C083E090E002C084E090E00E94E40880E090E008958FEF9FEF5C
:2016C000089581E090E00E942E080E94340A8038910521F184F48430910571F12CF40297A7
:2016E000A1F50E94C9082EC08031910511F1809761F50C94330B811522E0920791F034F485
:201700008115914011F582E090E010C0811524E0920751F08115984089F017C081E090E0B7
:2017200005C083E090E002C084E090E00E94E60009C00E94DB0806C00E94960880E090E0CF
:201740000E94FB0080E090E008958FEF9FEF0895FF920F931F93CF93DF9300D000D0CDB7F9
:20176000DEB78FEF9FEF9C838B839A838983FFB6F8940E941B0881E00E94180880E090E079
:201780000E941E08E0916C02F0916D020484F585E02D80E00995E0916C02F0916D0200884E
:2017A000F189E02D8EE692E009956EE471E08EE692E00E94900780915B01882339F08FEF9D
:2017C00099EF0197F1F700C00000DCCF01E010E00E94340A80329105E1F194F484309105F9
:2017E000C1F13CF49C01215031092230310580F730C08830910569F18031910549F729C0B8
:20180000811521E09207C1F04CF480349105E1F080389105E9F681E090E013C0811524E021
:20182000920769F0811528E09207E9F18115924079F683E090E005C082E090E002C084E03E
:2018400090E00E94FB0002C00E94610B019659F527C0AE014F5F5F4FBE016D5F7F4F0E94D9
:20186000B70A0196E9F08B819C810196C9F089819A810196A9F0012B21F080E090E00E94BA
:20188000FB0049815A816B817C8186E792E00E94C10581E090E00E942E0800E010E098CF98
:2018A0000E94510807C080E00E94180883E090E00E942E080E94E808FFBE0F900F900F906D
:2018C0000F90DF91CF911F910F91FF900895CF93DF931F92CDB7DEB70E94770490936D02D0
:2018E00080936C021AB88BB18B6F8BB9509A17B88FEF88B982E08093690091E09DBB10925A
:2019000055021092560210925702109258021092590210925A0210925B0210925C0295E010
:2019200090935D0210925E0280935F020E941B0881E090E00E942E080E94B208892B21F020
:2019400082E090E00E942E0878948091B60290E00E94FB000E947B08E0916C02F0916D0207
:201960000284F385E02D0995589A2FEF89E698E1215080409040E1F700C00000E0916C024E
:20198000F0916D020484F585E02D81E00995882329F0EFEFF9EF3197F1F7EECFE0916C0273
:2019A000F0916D020088F189E02D8EE692E009958FEF99EF0197F1F700C000008EE692E078
:2019C0000E944F066EE471E08EE692E00E94900780915B01882321F08EE491E00E94A80BED
:2019E00058980E94E80810E080916002882321F0109260020E94FA0880911C02882339F09B
:201A000080911C0290E00E94E60010921C020E944609882349F3589A0E946F08E0916C021D
:201A2000F0916D020484F585E02D80E0099589830E94750858988981882341F01F5F1531E4
:201A400034F081E090E00E942E0898CF10E0E0916C02F0916D020684F785E02D0995882337
:201A600071F1589AE0916C02F0916D020088F189E02D8EE692E009956EE471E08EE692E027
:201A80000E9490074AEB51E06EE471E086E792E00E94F20580916102882319F065E572E0C8
:201AA00002C069E572E08AEB91E00E9472019091610281E0911180E08093610258988EE40A
:201AC00091E00E94250190CF052E97FB1EF400940E947B0D57FD07D00E94A10D07FC03D088
:201AE0004EF40C947B0D50954095309521953F4F4F4F5F4F089590958095709561957F4FCD
:201B00008F4F9F4F0895A29FB001B39FC001A39F700D811D1124911DB29F700D811D112476
:201B2000911D08950E94830DB7FF0895821B930B0895B7FF0C94C30D0E94C30D821B930B2A
:201B40000895A1E21A2EAA1BBB1BFD010DC0AA1FBB1FEE1FFF1FA217B307E407F50720F07F
:201B6000A21BB30BE40BF50B661F771F881F991F1A9469F760957095809590959B01AC01F6
:201B8000BD01CF0108950E94830DA59F900DB49F900DA49F800D911D11240895FB01DC01EE
:201BA00004C08D910190801921F441505040C8F7881B990B0895FB01DC0102C001900D9275
:201BC00041505040D8F70895DC0101C06D9341505040E0F70895FB01DC0101900D9200201C
:201BE000E1F70895DC01CB01FC01F999FECF06C0F2BDE1BDF89A319600B40D92415050408B
:201C0000B8F70895DC01CB0103C02D910E940D0E41505040D0F70895262FF999FECF1FBA7F
:201C200092BD81BD20BD0FB6F894FA9AF99A0FBE01960895F894FFCF00000101020203035B
:201C40000404050506060707080809090A0A0B0B0C0C0D0D0E0E0F0F10141114121413140A
:201C60001414151416141714181419141A14FFFF0100080000000000000000006D0431048A
:201C80000203EE0265040100000001000000010000000100000001000000010000000300DD
:201CA000E000030020000300E0000300200001000000010000000100000001000000020015
:201CC00000000200000001000000010000000300E000030020000300E000030020000400F0
:201CE000200004002000020000000200000000000000010000000100000001000000010098
:201D00000000010000000100000001000000010000000100000001000000010000000100BB
:201D20000000010000000100000002000000020000000300810003007F0003008100030010
:121D40007F00000000004743324E36347638322E31005F
:0437FC0012345678B5
:203800000C94341C0C94431D0C94511C0C94511C0C94511C0C94511C0C94511C0C94511C6A
:203820000C94511C0C94511C0C94511C0C94511C0C94511C0C94511C0C94511C0C94511C20
:203840000C94511C0C94511C0C94511C0C94511C0C94511C0C94511C0C94511C0C94511C00
:203860000C94511C0C94511C11241FBECFEFD4E0DEBFCDBF11E0A0E0B1E0EEEAFEE302C004
:2038800005900D92A430B107D9F721E0A4E0B1E001C01D92A13BB207E1F70E946D1E0C94D8
:2038A000551F0C94001CF894299881E085BF15BEE0E0F0E0099408958130D9F48091890130
:2038C000813071F018F08F3F09F0DBC085E08093890110928A0182E080938B0183E008953C
:2038E0001092890110928A0110928B0110928C01A4C0823008F4C5C090918901923509F010
:20390000C0C090918A01913FD9F138F49130B9F008F4B8C0903F61F1B4C0993F09F496C017
:2039200020F4923F09F443C0ACC09E3F09F497C09F3F09F0A6C081E0809304019FC088E286
:20394000E9E8F1E0DF011D928A95E9F79093890180E880938A0188E380938B0110928C014B
:2039600060E071E083E991E00E944E1F8EE0089580918801811177C081E0809388017EC021
:2039800080918B0140918C0150E0582B60E070E0E5E0440F551F661F771FEA95D1F720E2F9
:2039A00030E089E891E00E94641E80E2089580918B0120918C0190918801911154C030E0A7
:2039C000382BA90143705527DA0185E0AA0FBB1F8A95E1F7A85FBE4F80E2EDE8F1E0019034
:2039E0000D928A95E1F7C901A0E0B0E062E0B695A795979587956A95D1F790930701809341
:203A0000060180910601909107019695982F88279795879590930701809306011092890104
:203A20004330510561F481E080938A0130938B0120938C0182E08093880184E00895109239
:203A40008A0130938B0120938C01F7CF9091880181E0911101C080E0809389010DC080913D
:203A60008801882321F081E08093890108951092890183E08093880181E008951092890111
:203A8000089580E008951F921FB64F930F931F93EF93FF937F93AF93BF93A9E8B1E00027CD
:203AA000EEEEFDE149B14470440F440F440F440F440F042B49B14470E9F31AE01A9521F08C
:203AC00049B14470D9F701C0099416E01A95F1F749B14470440F440F440F440F042B49B15A
:203AE0004470E9F31AE01A9521F049B14470D9F701C0099416E01A95F1F749B14470440F12
:203B0000440F440F042B49B14470E9F31AE01A9521F049B14470D9F701C0099416E01A950B
:203B2000F1F749B14470440F440F042B49B14470E9F31AE01A9521F049B14470D9F701C097
:203B4000099416E01A95F1F749B14470440F042B49B14470E9F31AE01A9521F049B1447019
:203B6000D9F701C0099416E01A95F1F749B14470042B49B14470E9F31AE01A9521F049B16F
:203B80004470D9F701C0099416E01A95F1F749B144704695042B49B14470E9F31AE01A95CB
:203BA00021F049B14470D9F701C0099416E01A95F1F749B1447046954695042B49B144704A
:203BC000E9F30D931AE01A9521F049B14470D9F701C0099415E01A95F1F761CF09E8A01B6B
:203BE00011F10F921F922F933F934F935F936F937F938F939F93AF93BF93FF938A2F11248D
:203C0000ECE5FCE10995082FFF91BF91AF919F918F917F916F915F914F913F912F911F9092
:203C20000F900DD000C0E09ABF91AF917F91FF91EF911F910F914F911FBE1F901895E9E8E4
:203C4000F1E0702F01D008953F937723D9F1772359F17A95019110E8302F312381F40000AB
:203C6000529A4FE04A95F1F700005298169579F3000000000000000000000000EDCF529AB9
:203C800044E04A95F1F70000000052984AE04A95F1F7000000001695D1F2000000000000F0
:203CA000000000000000D8CF00000000000000000000000000000000529A44E04A95F1F786
:203CC000000052983F910895FA01DC0102C005900D9221503040D8F70895CF93DF9300D0CE
:203CE00000D0CDB7DEB71AB88BEF8BB9509A17B88FEF88B9219A299881E085BF92E095BFEC
:203D0000909369008DBBF89424E030E040E050E0BA01CE0101960E94641E89818F3F61F46D
:203D20008A818F3F49F48B8111E08F3F31F48C818F3F19F410E001C011E024E030E04CEFA4
:203D400057E360E070E0CE0101960E94641E8981823151F48A81843339F48B81863521F442
:203D60008C81883709F496C080E0809305017894299A2FEF84E39CE0215080409040E1F702
:203D800000C00000299880910501882331F080910401811102C00E94531CC12CD12C7601E3
:203DA00013E001E0F5E0BF2EA1E1AA2EB2E09B2E80918801813051F008F451C08230E9F094
:203DC000833009F04AC00E94531C47C08FB7F894E0E0F0E0F999FECF07B600FCFDCF10932C
:203DE0005700E89507B600FCFDCFE058FF4FE11528E3F20779F78FBF30C04FB7F894F99918
:203E0000FECF07B600FCFDCF80E090E0FC01E85FFE4F2081FC01E75FFE4F5081E091060175
:203E2000F0910701E80FF91F30E0352B090100935700E895112402968038910539F7E0914D
:203E40000601F0910701B0925700E89507B600FCFDCFA0925700E8954FBF109288018091E7
:203E60000501811115C08FEFC81AD80AE80AF80A91EFC91699E4D90692E0E906F10408F492
:203E800097CF85B1892585B9C12CD12C760190CF299A8ECF81E0111168CF66CFFB01DC01F2
:123EA00001900D920020E1F70895F894FFCF312E300062
:0400000500003800BF
:00000001FF
